:020000040000FA
:08000000000000008801F32854
:08000800000020000D0880003B
:100010003F00E80A603068022000031918107608D3
:10002000970075089600111009008207003401340A
:1000300000340134003402348934C2348A34043444
:100040008934C434983428346B34C83400340034D0
:100050000034003400340034003400340034003400
:1000600000340034003400340034003400340134EF
:100070000034013400340234D134C234AA3404349C
:10008000A934C434883428348B34C8340034003460
:1000900000340034003400340034003400340034C0
:1000A000003400340034003400340034203481340F
:1000B0002034813420348234203482342034843417
:1000C000113404340A34083404340834003400345D
:1000D0000034003400340034003400340034003480
:1000E0000034003400340034003400340034003470
:1000F00004348034043400343434A2344C34A23414
:1001000044349434443494343C34883400340034DB
:10011000003400340034003400340034003400343F
:10012000003400340034003400340034FF348207DB
:10013000203434342034FF34313430342034FF342C
:10014000323430342034FF34353430342034FF340A
:100150002E343134203400342E3432342034003400
:100160002E343534203400342034313420340034FB
:1001700020343234203400342034353420340034F8
:1001800031343034203400343234303420340034CC
:1001900035343034203400343134303430340034A9
:1001A0003234303430340034353430343034003488
:1001B00082072E3431342E3432342E343534203408
:1001C0003134203432342034353431343034323424
:1001D0003034FB007B081520F900F90A03190800E8
:1001E000D923FB0AEA288C018D012100E1308C0023
:1001F000FF308D00F030990087309500013091007C
:10020000230001308C008D01210001309D00203041
:100210009E00250040309E0026002C309A000030C1
:1002200098009901280001309600171588012030A8
:10023000980065246524652465243030BA230C3089
:10024000BA230130BA23692469240630BA23023064
:10025000BA234030BA230030E920B323512274106E
:1002600074118C143430BA234C23F41A51233630D1
:100270007410BA23FF2116222030850084017208F1
:100280000319F82C013072020319BF2D02307202DB
:100290000319442F033072020319502F04307202E5
:1002A00003195C2F053072020319682F06307202A1
:1002B0000319762F073072020319842F0830720257
:1002C0000319922F093072020319A02F0A3072020B
:1002D0000319B12F0B3072020319BB2F0C307202BD
:1002E0000319C52F0D3072020319CF2F0E30720281
:1002F0000319D92F0F3072020319E32F87228921A6
:1003000074197F29741C862974103429FB0B7F29EA
:100310003C2921009D149D188B291C08FA00E63009
:100320001C0288010318A829F41CB52967242100A0
:100330009D149D1899291C08E6301C028801031899
:10034000080021001C0888017A02031D0800B72953
:10035000672421009D149D18AB291C08FA00E63083
:100360001C0288010318F4140800672408007414A0
:10037000F4101A307A02031CD1294E307A02031C81
:10038000DB2980307A02031CF929B4307A02031C7D
:10039000EC298C1E5F2A7419CF297415080074117A
:1003A0000800741908008C1AF229F419D929F415D7
:1003B0000800F4110800741908008C1AE529F41AD1
:1003C000E329F4160800F412080074190800F20A70
:1003D0000F30721AF200080074190800F203F21BC1
:1003E000F201080074190800F30A0730F319F3004A
:1003F000080074190800F303F31BF3010800073029
:10040000FB008C107B0873028C1103198C15082AD1
:100410008C147124FB0B012A8C100000F3088C1142
:1004200003198C1571248C14712408003230BA23FE
:10043000AB237208FA000310FA0DFA0D7A08972020
:10044000D923FA0A7A089720D923FA0A7A0897203A
:10045000D9232030D923AD237A0A9720FA0000301F
:10046000D923FA08003003190230D9230030D923E8
:100470000630D923AF237308FA000310FA0D7A0867
:10048000D820D9237A0AD820D923B1230030D92300
:100490000430D9230030D9230630D9233630BA238B
:1004A00008000030F0006D227108F200F00A6D22A1
:1004B0007108F300F00A6D227108F40008000030A2
:1004C000F0007208F1007522F00A7308F10075223D
:1004D000F00A7408F10075220800700823009100EA
:1004E000151413088801F100080071082300930017
:1004F0008801700823009100151555309600AA3028
:100500009600951415119518832A88010800F801A2
:100510002030850084010310800C0310800C840AB5
:1005200060300402031D8B2A84030008840A8000C3
:1005300020308500FF308400840A213087000C3091
:10054000860078083F3C00020319BB2A0318B12A31
:10055000840A78083F3C00020319B92A0318BA2A12
:10056000B92A840A78083F3C00020318B92A031408
:10057000BA2A03108403810D8603810D8603810D41
:100580008603810D8603810D8603810D8603810D0F
:100590008603810D8603810D8603810D8603810DFF
:1005A0008603810D5F300402031D9C2AF41EDA2AA3
:1005B000DF22DB2A1A23F80A781F982A0800213044
:1005C0008700013086003F3078020319EB2A0F3094
:1005D0007805031D042B01308104860A8104860AF4
:1005E0008104860A8104860A8104860A8104860AB7
:1005F0008104860A8104860A8104860A8104860AA7
:100600008104860A81041A2B07307805031D1A2BF2
:100610000130860A8104860A860A8104860A860ACF
:100620008104860A860A8104860A860A8104860A6B
:10063000860A8104F7017808803E9F39BA23823008
:10064000F81A8A307707BA232130870001308600F4
:100650000108D923860A0108D923860A0108D9236B
:10066000860A0108D923860A0108D923860A0108C7
:10067000D923860A0108D923860A0108D923860AC4
:100680000108D923860A0108D923860A0108D9233B
:10069000860A0108D9230800F8019823781F4D2BFA
:1006A0000800F8017B230730FB009823FB0B552B38
:1006B00063230730FB009823FB0B5B2B781F522B27
:1006C000F8037B230800F7017808803E9F39BA239E
:1006D0008030F81A88307707BA230030D9230030E9
:1006E000D923F70A0030D9230130D923F70AF71D9F
:1006F000722BF80A0800F7017808803E9F39BA2368
:100700008030F81A88307707BA230030D9230030B8
:10071000D923F70A0030D9230130D923F70A013051
:10072000D9230130D923F70AF71D8F2BF80A0800C7
:10073000F7017808803E9F39BA238030F81A883054
:100740007707BA230030D9230030D923F70AF71DE1
:10075000A22BF80A08008030BA2B9030BA2B8830D0
:10076000BA2B9830BA2B0130BA236924692402309D
:10077000BA230800F9008C15BD2B0C15BF2B0C11EA
:10078000C12B0C15C32B0C11C52B0C15C72B0C1131
:10079000C92B0C15CB2B0C11CD2B0C15CF2B0C1101
:1007A000D12B8C11D32B0C15D52B0C11D72B0C1551
:1007B000FA2BF9008C15DC2B0C15DE2B0C11E02B21
:1007C0000C15E22B0C11E42B0C15E62B0C11E82B6D
:1007D0000C15EA2B0C11EC2B0C15EE2B0C11F02B3D
:1007E0008C11F22B0C15F42B0C11F62B8C15F82B0D
:1007F0000C15FA2B0C11FC2B8C11FE2B0C15002C5C
:100800000C11F91B8C15042C0C15062C0C11082C42
:100810008C11791B8C150C2C0C150E2C0C11102C1A
:100820008C11F91A8C15142C0C15162C0C11182C73
:100830008C11791A8C151C2C0C151E2C0C11202CCB
:100840008C11222C0C15242C0C11262C0C15282C68
:100850000C112A2C0C152C2C0C112E2C0C15302CB8
:100860000C11322CF9198C15352C0C15372C0C1158
:10087000392C8C1179198C153D2C0C153F2C0C1131
:10088000412C8C11F9188C15452C0C15472C0C118A
:10089000492C8C1179188C154D2C0C154F2C0C11E2
:1008A000512C8C11532C0C15552C0C11572C0C154C
:1008B000592C0C115B2C0C155D2C0C115F2C0C159C
:1008C000612C0C11632C6F2C0800FA306A2C32302A
:1008D0006A2C0A30F1006F24F10B6B2C0800C73032
:1008E000722C1E30F0000000F00B732C080000008A
:1008F000792CF6308C2C00007D2C79308C2C00006B
:100900003B308C2C0000842C15308C2C00000930DE
:100910008C2C000000000330F0000000F00B8D2C48
:10092000080024007208C0007308C1007408C200E7
:100930008801080024004008F2004108F300420842
:10094000F4008801080021007008A0007108A100CF
:100950007208A2007308A3007408A4007508A5001B
:100960007608A6007708A7007808A8007908A900EB
:100970007A08AA007B08AB007C08AC007D08AD00BB
:100980007E08AE007F08AF008801080095010B11BA
:10099000F419D32C0B1908008D1FCA2C0B19080051
:1009A0008D1BCE2C08000B1908008D1BD32C0B19A6
:1009B00008008D1FD72C080095010B11F419EF2C9E
:1009C0000B1DE52CFB0BE52C08008D1FE02C0B1DEF
:1009D000EC2CFB0BEC2C08008D1BE72C08000B19F2
:1009E00008008D1BEF2C0B1908008D1FF32C08003D
:1009F0009124C6240D08A0000D08A1000D08A20036
:100A00000D08A3000D08A4000D08A5000D08A60000
:100A10000D08A7000D08A8000D08A9000D08AA00E0
:100A20000D08AB000D08AC000D08AD000D08AE00C0
:100A30000D08AF000D08B0000D08B1000D08B200A0
:100A40000D08B3000D08B4000D08B5000D08B60080
:100A50000D08B7000D08B8000D08B9000D08BA0060
:100A60000D08BB000D08BC000D08BD000D08BE0040
:100A70000D08BF000D08C0000D08C1000D08C20020
:100A80000D08C3000D08C4000D08C5000D08C60000
:100A90000D08C7000D08C8000D08C9000D08CA00E0
:100AA0000D08CB000D08CC000D08CD000D08CE00C0
:100AB0000D08CF000D08D0000D08D1000D08D200A0
:100AC0000D08D3000D08D4000D08D5000D08D60080
:100AD0000D08D7000D08D8000D08D9000D08DA0060
:100AE0000D08DB000D08DC000D08DD000D08DE0040
:100AF0000D08DF000D08E0000D08E1000D08E20020
:100B00000D08E3000D08E4000D08E5000D08E600FF
:100B10000D08E7000D08E8000D08E9000D08EA00DF
:100B20000D08EB000D08EC000D08ED000D08EE00BF
:100B30000D08EF000D08F0000D08F1000D08F2009F
:100B40000D08F3000D08F4000D08F5000D08F6007F
:100B50000D08F7000D08F8000D08F9000D08FA005F
:100B60000D08FB000D08FC000D08FD000D08FE003F
:100B70000D08FF00A3249A243230FB007E29912423
:100B8000C6240D08A000C42D00000D08A100C82D2A
:100B900000000D08A200CC2D00000D08A300D02DF0
:100BA00000000D08A400D42D00000D08A500D82DCC
:100BB00000000D08A600DC2D00000D08A700E02DA8
:100BC00000000D08A800E42D00000D08A900E82D84
:100BD00000000D08AA00EC2D00000D08AB00F02D60
:100BE00000000D08AC00F42D00000D08AD00F82D3C
:100BF00000000D08AE00FC2D00000D08AF00002E17
:100C000000000D08B000042E00000D08B100082EF1
:100C100000000D08B2000C2E00000D08B300102ECD
:100C200000000D08B400142E00000D08B500182EA9
:100C300000000D08B6001C2E00000D08B700202E85
:100C400000000D08B800242E00000D08B900282E61
:100C500000000D08BA002C2E00000D08BB00302E3D
:100C600000000D08BC00342E00000D08BD00382E19
:100C700000000D08BE003C2E00000D08BF00402EF5
:100C800000000D08C000442E00000D08C100482ED1
:100C900000000D08C2004C2E00000D08C300502EAD
:100CA00000000D08C400542E00000D08C500582E89
:100CB00000000D08C6005C2E00000D08C700602E65
:100CC00000000D08C800642E00000D08C900682E41
:100CD00000000D08CA006C2E00000D08CB00702E1D
:100CE00000000D08CC00742E00000D08CD00782EF9
:100CF00000000D08CE007C2E00000D08CF00802ED5
:100D000000000D08D000842E00000D08D100882EB0
:100D100000000D08D2008C2E00000D08D300902E8C
:100D200000000D08D400942E00000D08D500982E68
:100D300000000D08D6009C2E00000D08D700A02E44
:100D400000000D08D800A42E00000D08D900A82E20
:100D500000000D08DA00AC2E00000D08DB00B02EFC
:100D600000000D08DC00B42E00000D08DD00B82ED8
:100D700000000D08DE00BC2E00000D08DF00C02EB4
:100D800000000D08E000C42E00000D08E100C82E90
:100D900000000D08E200CC2E00000D08E300D02E6C
:100DA00000000D08E400D42E00000D08E500D82E48
:100DB00000000D08E600DC2E00000D08E700E02E24
:100DC00000000D08E800E42E00000D08E900E82E00
:100DD00000000D08EA00EC2E00000D08EB00F02EDC
:100DE00000000D08EC00F42E00000D08ED00F82EB8
:100DF00000000D08EE00FC2E00000D08EF00002F93
:100E000000000D08F000042F00000D08F100082F6D
:100E100000000D08F2000C2F00000D08F300102F49
:100E200000000D08F400142F00000D08F500182F25
:100E300000000D08F6001C2F00000D08F700202F01
:100E400000000D08F800242F00000D08F900282FDD
:100E500000000D08FA002C2F00000D08FB00302FB9
:100E600000000D08FC00342F00000D08FD00382F95
:100E700000000D08FE003C2F00000D08FF00A32419
:100E80009A243230FB007E296030FB00C6240D0816
:100E900080009024840AFB0B472F3230FB007E2910
:100EA0006030FB00C6240D0880008924840AFB0BF7
:100EB000532F3230FB007E296030FB00C6240D0822
:100EC00080008624840AFB0B5F2F3230FB007E29D2
:100ED0000230FB00DC246030FB000D08800082241F
:100EE000840AFB0B6D2F3230FB007E290330FB00A0
:100EF000DC246030FB000D0880007F24840AFB0B9B
:100F00007B2F3230FB007E290430FB00DC24603074
:100F1000FB000D0880007B24840AFB0B892F3230F4
:100F2000FB007E290530FB00DC246030FB000D084F
:100F300080007724840AFB0B972F3030FB007E293A
:100F40000630FB00DC246030FB000D0880007724B5
:100F500077247B248A24840AFB0BA52F2C30FB00EA
:100F60007E29FB30F6002030F5000A30FB00ED272B
:100F70000130FB007E29F630F6003E30F5000A30E5
:100F8000FB00ED270130FB007E29E730F6009830AA
:100F9000F5000A30FB00ED270130FB007E29CF3041
:100FA000F6002E30F5000A30FB00ED270130FB0083
:100FB0007E299E30F6005A30F5000A30FB00ED27FE
:100FC0000130FB007E290B30F600DE30F5000A30E0
:100FD000FB00ED270130FB007E29FF3097009600D3
:100FE00011100B17DC248B17181489217418FA2F91
:0C0FF0001818F52F8B130B1318100800B5
:040FFC000034003489
:020000040001F9
:02000E00820965
:02001000FF1DD2
:06E000000A0001002000EF
:00000001FF
